S01A0000666C6173686C6F616465725F6C6F616465722E73726563AF
S11300000020002011040000073200000732000025
S11300100732000007320000073200000000000031
S11300200000000000000000000000000732000093
S11300300732000000000000073200000732000011
S11300405D3300005D3300005D3300005D3300006C
S11300505D3300005D3300005D3300005D3300005C
S11300605D3300005D3300005D3300005D3300004C
S11300705D3300005D3300005D3300005D3300003C
S1130400FFFFFFFFFFFFFFFFFFFFFFFFFEFFFFFFF9
S113041072B60E480E49886000220023002400258D
S113042000260027B846B946BA46BB46BC4609482A
S1130430854609488047094880470948804762B68D
S113044000200021074A9047FEE70000000000005A
S113045000ED00E000200020053300000932000018
S113046043320000B104000072B60D490020086058
S1130470BFF36F8FBFF34F8F704780B542F6D842FA
S11304800FF23401074802F093FEFFF7EDFF064830
S113049080F3088880F309880448BDE802400047D7
S11304A008ED00E000E0FF1FA811002011E4FF1F89
S11304B080B5FFF7E2FFFEE7A811002011E4FF1F5B
S11304C0EBE4FF1F31FCFF1F33FCFF1F35FCFF1F54
S11304D037FCFF1F000000000000000000000000C7
S11304E000000000EBE4FF1FEBE4FF1F000000002E
S11304F0EBE4FF1F83E8FF1F790C0020790C002038
S1130500790C0020790C0020790C0020790C002053
S1130510790C0020790C0020790C0020790C002043
S1130520790C0020790C0020790C0020790C002033
S1130530790C0020790C0020790C0020790C002023
S1130540790C0020790C0020790C0020790C002013
S1130550790C0020790C002017020020790C00206F
S1130560EDFDFF1F790C0020790C0020790C002090
S1130570790C002013070020790C00201F070020AD
S1130580790C0020790C0020790C0020790C0020D3
S1130590790C0020790C0020790C0020790C0020C3
S11305A0790C0020790C0020790C0020790C0020B3
S11305B0790C0020790C0020790C0020790C0020A3
S11305C0790C0020790C0020790C0020790C002093
S11305D0790C0020790C0020790C0020790C002083
S11305E0790C0020790C0020790C0020A7E9FF1F6A
S11305F0790C0020790C0020790C0020790C002063
S1130600790C0020790C0020790C0020790C002052
S1130610790C0020790C0020790C0020790C002042
S1130620790C0020790C0020790C0020790C002032
S1130870790C0020790C0020FFFFFFFFFFFFFFFF32
S1130880FFFFFFFFFFFFFFFFFFFFFFFFFFFFFFFF74
S1130890FFFFFFFFFFFFFFFFFFFFFFFFFFFFFFFF64
S11308A0FFFFFFFFFFFFFFFFFFFFFFFFFFFFFFFF54
S11308B0FFFFFFFFFFFFFFFFFFFFFFFFFFFFFFFF44
S11308C0FFFFFFFFFEFFFFFF72B60E480E49886070
S11308D0002200230024002500260027B846B9463C
S11308E0BA46BB46BC46094885460948804709487C
S11308F080470948804762B600200021074A904794
S1130900FEE7000000E0FF1F00ED00E0A81100205A
S1130910C10A002069F7FF1FA3F7FF1FE1F1FF1FC2
S11309200000000000000000002A01D101207047EF
S1130930F0B41F46034603242340002B09D00424AB
S1130940E31A017001300824E141521E26D05B1ED7
S1130950F7D1042A1ADB13D0002F11D00C460D4610
S11309600E46102A02DB72C0103AFAE70C2A02DBA8
S113097032C00C3AFAE7082A02DB12C0083AFAE756
S1130980042A03DB01600430121FF9E7002A05D0B2
S1130990017001300824E141521EF7D1F0BC00205F
S11309A07047FEE781EBFF1F0000000093EBFF1F81
S11309B0000000000000000000000000F1EBFF1F39
S11309C045ECFF1F000000000000000000000000D4
S11309D000000000A7EBFF1F000000000000000063
S11309E000000000E9ECFF1F000000000000000010
S11309F00000000037EBFF1F00000000DBEBFF1FCF
S1130A0000000000000000000000000000000000E2
S1130A1000000000000000000000000000000000D2
S1130A2000000000000000000000000000000000C2
S1130A30000000000001024669F2FF1FBDF2FF1F23
S1130A4000000000DFF2FF1F65F3FF1FE9F3FF1F43
S1130A5019F4FF1F7BF4FF1F87F4FF1F0FF5FF1F1F
S1130A6015F6FF1F00000000000000000000000059
S1130A70000000000000000093F5FF1F00000000CC
S1130A800000000000000000000000000000000062
S1130A90650C00206F0C0020000000000000000026
S1130AA000000000B1FCFF1FF3FCFF1F4BFDFF1F04
S1130AB000000000000000007FFDFF1F69EEFF1F23
S1130AC099EEFF1FD9EEFF1F000000000000000098
S1130AD099EFFF1F79020020B90200205F03002074
S1130AE000000000000000009B030020B5FAFF1F77
S1130AF06DF9FF1F95F9FF1F000000001FFAFF1F8B
S1130B00D1F9FF1F9FF8FF1FA3F8FF1FB5F8FF1FC0
S1130B1000000000000000000000000001000000D0
S1130B2001000000F3E8FF1FD8E6FF1FE8E6FF1FFF
S1130B30F0E6FF1F020000000000000037E9FF1F7D
S1130B401CE6FF1F2CE6FF1FF0E6FF1F0400000059
S1130B500000000063E9FF1FECE5FF1FFCE5FF1F39
S1130B60F0E6FF1F0000000000000000000000008D
S1130B70000000000000000000000000C903002085
S1130B800704002019050020CD050020480E002090
S1130B9039060020B3060020CD0600200000000026
S1130BA000000000FF0600207107002077070020E6
S1130BB0DF0700207D080020750700208908002039
S1130BC05107002038B504463D4D0020C5E900001A
S1130BD0C5E90200C5E9040028626862394800F0EA
S1130BE0A0F8C5E906012046BDE834400FF25501DE
S1130BF000F046B900F056B970B5314D0C46296A7B
S1130C00072904BF696A88421AD100F093F8C0EB3F
S1130C100016D5E90001D5E902231018B6FBF0F05F
S1130C200A2148434FF49661B0FBF1F0401D0A21BC
S1130C30B0FBF1F04FF4966148432060002070BD92
S1130C40012070BD2DE9F843064600F05AF81C4F08
S1130C500446386AD7E904598846421CD7E9060194
S1130C60651B68EB0909494502D82CBFA84201223B
S1130C70012A3A6206D0042A08D0052A0ED0072A8F
S1130C800FD018E0C7E900487E6214E0D7E90001FC
S1130C90201A68EB0101C7E900010CE0C7E902482A
S1130CA009E0D7E90201201A68EB0101C7E9020152
S1130CB0304600F0F7F8C7E90448BDE8F1830000C6
S1130CC0D00D0020803801001E48002101606FF023
S1130CD07F421D494A6000228A6007220A601B493C
S1130CE01B4A0968C900B1FBF2F101B90121416055
S1130CF0704715480168C908C90001600021816076
S1130D00704710490A68134800680B68C043000222
S1130D10000A9A42F6D1002110EB026051EB122135
S1130D20704708494968A1FB0001C00840EA4170C6
S1130D30C908704705480068704702480168491CA3
S1130D4001607047380E002010E000E0CC0D002058
S1130D5040420F0018E000E00901002806D55D4A72
S1130D6000F00F00801800F8041C70475A4A8154A0
S1130D70704750F82130120423F4702302F47022D7
S1130D801A430FE050F82100C0F30060704706E0FA
S1130D90120202F4E06242F0200203E000BF1202F9
S1130DA002F4E06240F821207047012800D0704727
S1130DB010B54A4C19B102290ED004D310BD00203D
S1130DC0E060206110BD4FF48070E0604448016829
S1130DD021F00801016010BD032203212046FFF722
S1130DE0D6FF2046BDE8104003220421CFE700B11E
S1130DF0704710B53B4C11B1022903D010BD2060DF
S1130E00606010BD022201212046FFF7C1FF204689
S1130E10BDE8104002220021BAE700B1704710B5C6
S1130E20314C11B1022905D010BD20646064A06466
S1130E30E06410BD022210212046FFF7AFFF02221A
S1130E4011212046FFF7AAFF022212212046FFF7B4
S1130E50A5FF2046BDE81040022213219EE780B57D
S1130E6003211E48FFF78EFF48B12048416808005F
S1130E7005D0012088471E494FF0FF30086001BDAE
S1130E8010B501280C460CD101213D20FFF764FF69
S1130E9018494FF0005008600A2200F016F8134871
S1130EA0446010BD012800D0704780B512494FF04E
S1130EB00050086000213D20FFF74EFF002200F0A3
S1130EC004F80A490020486001BD0321034850E7A3
S1130ED00000000018ED00E000E400E000B0044071
S1130EE094F00F4000A0044000D00440400E0020C5
S1130EF0A0B0044004E100E084E100E0DFF8A413C2
S1130F00C968C9680020086070472DE9F041DFF81E
S1130F10945382B0E86900248DF801404669002E9C
S1130F2062D0E968C9680A68012A4CD001F1080254
S1130F3074680023091DA04704001FBF42F2127009
S1130F40844242F2137084424ED1E868C168D1F8F9
S1130F500880B8F1000F47D04E68377837B1132FA7
S1130F6004DA806800EBC700083800E0002008625B
S1130F7000281CBF006800281CD02A6992696946B1
S1130F8005F120009047040016D19DF8000040B1FF
S1130F904FF4E750791EC840C00758BF42F211749D
S1130FA00AD5EA68D268126A126841463046904708
S1130FB0002406E042F210743946204600F028F975
S1130FC094B901200DE0086A48B14168080003D0D3
S1130FD00DF10100884704460CB1002001E09DF8A2
S1130FE00100E968C96808602046BDE8F68180B55B
S1130FF00178002000F00CF9DFF8A802C06941690B
S113100009698847022000F055F9BFF34F8FDFF8D4
S11310109802DFF89822016801F4E061114301604D
S1131020BFF34F8F00BFFDE7DFF87802C068C068E8
S113103014210C3000F070B910B5044600F023FA06
S1131040FFE72178BDE81040E2E010B5DFF8542254
S1131050126852690446A16860689047F1E730B5A8
S113106083B0DFF84042A5680021019100916B46EE
S113107081684068AD6801AAC9B2C0B2A847E268F5
S1131080D2680021116100998A08019900F0D4F80E
S113109037BD10B5DFF80C229268D2680446606848
S11310A0A168C0B29047CCE710B500F006F800F094
S11310B006F8042101770020C3E70446B4E7DFF80B
S11310C0E401C068C068A16801616168416170475A
S11310D038B5DFF8D0510446E868C06800214161A2
S11310E00161007F042804D128680069804704B99D
S11310F00446E868C068017F204686E02DE9FC418B
S1131100DFF8A0610446F068C068016921B90020D5
S11311102070FFF7DDFF40E0012121700569476978
S1131120002000900123F069D0F814C0DCF804C05A
S11311306A4601A9E0475FEA000805D0F069416901
S1131140C9688847404603E0009830B942F21270FB
S1131150FFF7BEFF0020207020E0A84288BF284689
S11311603368019A009001469B6838469847804648
S11311700098C7192D1A06D0B8F1000F09D0F069EC
S11311804169C96888474046FFF7A2FF00202070E4
S113119003E0F068C068056147610020BDE8F6819E
S11311A02DE9F0410546424C6E68D5F80880E868A0
S11311B03C49206000274968103130B10A689042E8
S11311C023BF4968491C81420427304600F0D0F906
S11311D000B904272978384600F01AF89FB96660E8
S11311E0002000F067F82068C4F8088018B180F384
S11311F0088880F30988616840468847BDE8F04163
S1131200002000F057B8BDE8F081BDE83440FFE7A6
S113121010B584B0A02201908DF80020002200F0C7
S11312203BF88DF80220029102228DF8032000235E
S11312304469A4680C222CE010B588B0A72300F000
S11312401FF80020531C8DF8033006E06C4651F85B
S1131250203004EB8004401CA3609042F6D300F0DD
S113126006F80023FFE76946A04708B010BD0D4803
S1131270C0699DF803104469A46889000A1D704779
S11312808DF80030019000238DF801308DF8023084
S113129070476946A0471FBD0248C0698DF8012008
S11312A070470000E80C00200CED00E00400FA0593
S11312B01C0E002070B50446022C04D0002000F05F
S11312C040FC012C0ED00026114D06E04019C168E7
S11312D089680A0018BF8847761C18207043415952
S11312E00029F3D174B900F093FCFFF702FD00F07C
S11312F0B4FC084900200860012000F0DBFC00F089
S1131300E4FC62B6BFF36F8FBFF34F8F70BD00BFB5
S113131064E6FF1F08ED00E0002200F003BD0000BA
S113132038B5844D2B696C68DB6A2246042105F1CB
S1131330200098472B69DB6A6A46012105F12000E9
S11313409847206800990818401E6060002032BD4C
S1131350F8B5784F0446786B0D464042164600EACD
S11313600401621AAA1852421040424207F12000B6
S11313703F697F6C6B46B84748B99DF8000008B1D7
S11313806C20F2BD32462946204600F0E6FCF2BD50
S11313902DE9F04389B0914604460F4603AA00F0B4
S11313A0B1F8002846D1BE08B600BF1B4FF0FF308D
S11313B00690079005D03A4606EB090106A800F00E
S11313C0F5FC06EB04085B4D56B1D5F810C0DCF80B
S11313D014C033464A46214605F12000E04750B97F
S11313E057B1D5F810C0DCF814C0042306AA41464E
S11313F005F12000E047E8B99DF80C00C8B15EB1E2
S113140004A80290214605A801904B4600F015F867
S1131410324600F018F858B95FB104A8029006AB40
S113142005A80190082200F008F8414600F00BF8E6
S113143000B9002009B0BDE8F083A8680069006D18
S1131440C0B2009070472C69A46A05F120002047BF
S1131450F8B504460D46374E374B37693F692A467F
S1131460214606F12000B84760B9B16809690A6BE2
S113147042B10B6D21463469646ADBB22A4606F137
S11314802000A047F2BD10B52A4C2B49226992686E
S113149004F12000904758B9A16809690A6B22B188
S11314A02269096D00F029F810B9244A012111704C
S11314B010BD70B5154682B000222A700A461D4C34
S11314C02669766C01466B4604F12000B04798B952
S11314D09DF8001029709DF8001069B1174D297806
S11314E051B9A06800692269016D00F006F808B1DD
S11314F06C2076BD0121297076BD126AC9B204F14F
S11315002000104710B514460A4A82B09268126946
S1131510126B02B1012249422270890889006A468D
S11315204942FFF7C6FF20B99DF8001009B1002118
S1131530217016BDE80C00206B66656BA00F0020BF
S113154038B504460D460020FFF7B4FE6E486F4AD6
S11315500560446000211160016881F3088881F30B
S1131560098840688047BDE832400020FFF7A2BEEA
S113157010B582B000281EBF10F1010F64498842E3
S113158001D1002016BD6A46022100F0B0FC0024FF
S113159018B90098007A00B10124204616BD2DE93F
S11315A0FC47DFF870815C4DD8F80800006900F151
S11315B068072E4609E0397C014205D07069F2685B
S11315C08169526830469047183630680028F2D155
S11315D00024A146CDE900494FF47A70FFF7A1FB3E
S11315E006468A4600F096FBA0BBFFF7C1FF88B30E
S11315F0D8F80800006990F88600C00703D40021D9
S11316000020FFF79DFF788A4FF6FF71884208BFDC
S113161041F28830A6FB00230AFB0033CDE9002306
S1131620FFF76FFB04468946DDE90001002908BF86
S113163000280FD0FFF765FBDDE90023001B61EBF9
S11316400901994206D301D8904203D30021002016
S1131650FFF776FF2E4600E0183630680028E3D006
S1131660397C0142F8D0F16809683046884700287F
S1131670F2D0002ED8D009E0397C014218BFAE4226
S113168003D0E968896828468847183528680028FF
S1131690F2D13046BDE8F68738B500F0B3FA00F071
S11316A00BFB1C4C2169496804F120008847A068A1
S11316B000688047002000F0FDFAFFF705FB206872
S11316C000688047A06840688047FFF768FFE061D2
S11316D0016919B109680A0018BF8847E0694169BE
S11316E019B109680A0018BF8847E0680068804794
S11316F0E569E06840688047E868C1680800F8D098
S113170028468847F5E70000280E002008ED00E091
S113171011E4FF1FE80C002064E6FF1F704700007F
S113172008B904207047DFF830140968090E01F085
S11317300F010F290FBF4FF400310FF2A84232F806
S1131740111089020022026041604FF4807201216D
S113175081604FF40061C160DFF8001491F900303A
S11317609A404261C978816100210161016241624C
S11317700020704738B5040001D1042032BDDFF8E1
S1131780E0236FF03B401060DFF8D803814201D0C2
S11317906B2032BD38E02DE9F04389B0164680460F
S11317A00D4600F04AF9049B00F043F904001BD1F4
S11317B0009D019F7019461EB6FBF7F007FB1061F0
S11317C021B1401C7843461E00E07D19AE4217D378
S11317D02802000ADFF8881340F010600860DFF880
S11317E08403814502D06B24204656E000F0E9F8DA
S11317F00446D8F81000010018BF8047002CE4D03C
S1131800404600F09EF9EFE7204600F084F900F02E
S113181002F8284632BD0546204692E12DE9F04300
S113182089B004465FEA02080F461D4608BF04203B
S113183033D000F003F9039B2A463946204600F0D2
S11318409DF95FEA000928D1009FDFF8146302E0E4
S11318500398C7192D1AEDB158F8040B70603902BA
S11318600398090A042808BF41F0C06006D008287C
S113187005D158F8040BB06041F0E06030602046B8
S113188000F049F981462069010018BF8047B9F189
S1131890000FDDD0FFF7C0FF484609B0BDE8F08374
S11318A0002818BF002901D104207047DFF8B802CE
S11318B0007800F00302022A08BF002005D000F0DF
S11318C0C00080280CBF012002200870002070474F
S11318D010B50A46002818BF002A01D1042010BD03
S11318E0DFF884321C78002104F00304022C1ED09B
S11318F06FF03A41C3F8021054781178240444EA92
S11319000161947841EA0421D4782143C3F8061094
S113191054791179240444EA01619479D27941EA31
S113192004211143C3F80A1000F0F5F801460846F3
S113193010BD08B904207047DFF8302280E02DE99B
S1131940F04F89B0924680460C4600F076F8059B2D
S113195052462146404600F011F978BB6A462146BA
S1131960404600F020F9009C029E6042714208400B
S11319704542A54208BF7519794F03E0AAEB0B0A4B
S11319805C447519BAF1000F17D0281BD346824561
S113199088BF83460598BBFBF0F02102090A0004C6
S11319A041F0807140EA0920396040F0FF0078601E
S11319B000F007F80028E1D000E0002009B0BDE8FD
S11319C0F08F4046A7E02DE9F04389B080465FEAF6
S11319D003090D46164608BF042029D000F02EF84E
S11319E0079B00F026F818BB009D109C5C4F05E097
S11319F007998A08761A09EB82094D19C6B128029B
S1131A00000A40F000703860200640F0FF1040F4F7
S1131A107F407860D9F80000B860FFF7D2FF002853
S1131A20E6D0119901B10D60129909B100220A6042
S1131A3033E7324629464046A0E099466A46B2E07A
S1131A4042EA0141464A116065E02DE9F0418046D1
S1131A501E000D46174608BF042034D0042300F0AE
S1131A608DF880BBD8F814307A195F42C2F1000CAB
S1131A7007EA0C0CCCF1000C2F40ACEB070700215B
S1131A80B7FBF3F7DFF8E8C00AE0DCF800E0203C3D
S1131A906FEA0E0E2EFA04F4E40748BF491C5D19E0
S1131AA095420AD2B5FBF3F4202C38BFDCF804E0ED
S1131AB0EED3D8F818E07445E7D319B1B94234BF6E
S1131AC0022101213170BDE8F0810000002818BF17
S1131AD0002A01D10420704709291AD8DFE801F04F
S1131AE00509090B0D0F11131517C06810600020AC
S1131AF070474068FAE78068F8E70068F6E7012075
S1131B00F4E74069F2E78069F0E7006AEEE7406ACB
S1131B10ECE76A207047174870210170802101703A
S1131B2001780906FCD50078810601D56720704745
S1131B30C10601D568207047C0074CBF692000204A
S1131B4070470D49096851F470010B4A1160BFF3E5
S1131B506F8FBFF34F8F70474C80044028000240C2
S1131B60040002406B66656B02000240FFFF004008
S1131B70180002400000024004F0014008B90420AB
S1131B8070475B1E194208BF1A4201D06520704796
S1131B900368994221BF4068C0185118884234BF75
S1131BA066200020704770B505000E46144601D12A
S1131BB0042070BD20212046FFF7AEFB2868301AB0
S1131BC02060E8686060A9686868B0FBF1F0A06014
S1131BD00420E0600820206160610420A061E061CD
S1131BE0002070BD080010001800200030004000E4
S1131BF060008000C00000018001000200030004B6
S1131C000006000072B605490020086062B67047FD
S1131C1072B602480168491C01607047300E00200A
S1131C2080B518491848086018491948421A1948D3
S1131C3088421CBF002A00F0B9F817481749091A4E
S1131C4018BF00F0A5F916491648421A04D0BDE899
S1131C500840154800F0AAB801BD14484FF0FF3100
S1131C60016041608160C160016141618161C16164
S1131C700F48016041608160C1600161416181611F
S1131C80C161704708ED00E000E0FF1F240B002055
S1131C901C0C0020D80C0020D00D0020A40F002024
S1131CA0D80C0020D80C0020A40F002080E100E014
S1131CB080E200E07047000080B500F06DF9124842
S1131CC0016841F47851016001BD0F48016821F4B5
S1131CD07851016070470D480D4A01680068126828
S1131CE0000F401CC1F303615043491CB0FBF1F0E9
S1131CF07047012802D0022803D003E0044800689A
S1131D007047E8E70020704738800440448004406E
S1131D10CC0D0020002070477047000062F30F22B2
S1131D2062F31F4200B500BF130096469446103973
S1131D3028BFA0E80C50FAD85FEA417C28BF0CC049
S1131D4048BF40F8042BC90728BF20F8022B48BF1E
S1131D5000F8012B00BD00F037B9134680B50A46E0
S1131D600146184600F022F8002002BD70B510F0BC
S1131D70030F0C46154612D0B0F1005F0FD22118A4
S1131D80491EB1F1005F0AD3C0F10056324629461C
S1131D9000F00CF8A21B71194FF0005001E022462C
S1131DA0294600F003F8002070BD000062B38B07E1
S1131DB008D0521E11F8013B00F8013B00F02480CA
S1131DC08B07F6D1830740F0208000BF103A07D379
S1131DD030B4B1E83810103AA0E83810F9D230BC69
S1131DE0530724BFB1E80810A0E8081044BF51F815
S1131DF0043B40F8043BD20724BF31F8022B20F8FF
S1131E00022B44BF0B7803707047083A07D3B1E83C
S1131E100810083A40F8043B40F804CBF7D25307C3
S1131E20E4E7000070B50D0082B00446164601D107
S1131E30002076BD6A4600F05AF830B9009BDB6892
S1131E405B68324629462046984776BD70B50D003A
S1131E5082B00446164601D1002076BD00F068F831
S1131E6000B135E000F030F868B9009BDB689B688E
S1131E7032462946204698474349002806BF009A1F
S1131E80D26800220A6076BD38B504460D466A461B
S1131E9000F02DF8A0B90098C068406908B9662020
S1131EA032BD2946204600F043F810B142F2D87002
S1131EB032BD009AD268526929462046904732BD05
S1131EC0002DFCD1002032BD6A46294620460EE092
S1131ED042F2D87076BD10B52B4C2168002029B190
S1131EE009690A0002D088470021216010BD70B53D
S1131EF042F2D873D2B1254C6468146011B915E06C
S1131F001034146014688CB12568002D04BF666811
S1131F10002E01D1E6684EB1A84224BF656885420F
S1131F20EED30818401E854228BF0023184670BD12
S1131F3070B50918491E0022144B9C685D68246919
S1131F40160104EBC2045834755966682468AC421F
S1131F5008BFAE4205D0864228BFA14201D301206A
S1131F6070BD521C022AE8D3002070BD10B507488A
S1131F70446804E00068010018BF80471034E0683A
S1131F800028F7D110BD0000340E0020E80C00201A
S1131F90002200F059B800000948817804290DD1C5
S1131FA0017801F09F010170FF218278012A03D199
S1131FB0044A1278520701D4491EF6D17047000032
S1131FC001E0074002D007401D480068000B00F004
S1131FD00F00C01E082830D8DFE800F005080B0EFB
S1131FE01114172F1A004FF4804013E04FF4C0402F
S1131FF010E04FF400400DE04FF440400AE04FF48D
S1132000803007E04FF4C03004E04FF4003001E0CA
S11320104FF480200121421E10420A4A18BF0221B7
S113202052684B1CB0FBF3F0C0F1005342F8103F70
S11320306FF0604301FB003050600020704700BF28
S113204000700440E80C0020401810F0030308D08E
S1132050C91A1FD3DB0748BF00F8012D28BF20F899
S1132060022D130030B414461546103928BF20E958
S11320703C00FAD8490728BF20E90C0048BF40F8C3
S1132080042D890028BF20F8022D48BF00F8012D37
S113209030BC7047C91818BF00F8012DCB0728BF02
S11320A000F8012D7047000030B901290CBF034925
S11320B003494FF080600860704700BF00E100E012
S11320C080E100E0BFF34F8F0548064A016801F440
S11320D0E06111430160BFF34F8F00BFFDE70000D3
S11320E00CED00E00400FA05ECE7EBE7EAE7E9E7CA
S11320F030B901290CBF034903494FF080700860CF
S1132100704700BF00E100E080E100E010B582B05C
S113211000228DF800200A46064C014604F12000F6
S11321202469646C6B46A0479DF8000000B101204F
S113213016BD0000E80C002001280ED80FF224027E
S113214080560122012900F01F0102FA01F10CBF9F
S1132150024A034A400942F82010704700E100E0B7
S113216080E100E01F21000040684A49405C70475C
S113217048498A6842B14A6813780370501C486021
S11321808868401E886070470021017070475A2893
S113219007D1404A01238B540FF20901116151699F
S11321A0084770473B49496908477FB5394D69611C
S11321B004460FF2F400616850F82160684600F0AC
S11321C0DFF801208DF808008DF80900022132485B
S11321D0E86032482861A2686068904769463046E2
S11321E000F084F82E49304600F0FCF860680121C4
S11321F0FFF75AFF616849190120487004B00020B4
S113220070BD70B50546234C68680119497889B1D9
S11322100FF2940151F820600021FFF745FF30468A
S113222000F0BAF86868AA6800219047696809193B
S11322300020487070BD17484160826081680029A1
S1132240FCD10020704770B504460FF25C0082B0E8
S113225050F82450E86A00010BD54FF0006007E005
S1132260F168684688479DF8000068634FF0007085
S1132270E862E86A074E8001F2D4E86A800308D570
S1132280A86B4FF40031E96221463269C0B290472D
S1132290F3E773BD3C0D0020B9FCFF1FD7FCFF1F03
S11322A00000020A0020CEE700C00240010C01F148
S11322B0804101F58E2101230A6803FA00F01043DE
S11322C0086070470029016814BF21F4804141F47B
S11322D08041016070470021DFF83821904218BF27
S11322E001210846704701212046EBE738B5044632
S11322F00D46FFF7F0FF00F03EF8FFF7F4FF00F0A3
S113230083F80122206840004008206020680840CB
S1132310297B40EA8170A97B40EA8160697B40EABD
S11323200160E97B00F01CF80121204600F04FF821
S1132330287804EB8000C1686A6821F0FE41521ECF
S113234041EAC2612A7A920602F0806211436A7AF3
S1132350520602F000721143C16000F007F831BD6B
S1132360090201F440710843206070472068400866
S11323704000206070470FF2A40151F8200095E757
S11323800021017008214160002101724172017332
S113239041738173C173704710B5044600212068EE
S11323A000F034F8FFF7A0FF00F02CF80FF26C01F6
S11323B051F82000010C01F1804101F58E21012327
S11323C00A6803FA00F022EA0000086010BD0368FE
S11323D0090401F47C11012A0CBF194323EA010109
S11323E0016070478A0103D5026B22F08072026398
S11323F08A0303D5026B22F480320263026B114319
S113240001637047204666E72068034940F00100F5
S11324102060704700C00240FFCCFFBA0C003C10A3
S1132420010C01F1804101F58E2101230A6803FAB0
S113243000F0104308607047010C01F1804101F580
S11324408E2101230A6803FA00F022EA00000860E2
S113245070470029817814BF41F0800101F07F01A9
S1132460817070470021DFF8E820904218BF0121F5
S1132470084670474A0603D5827842F040028270CB
S1132480890603D5817941F0200181717047C178B3
S11324908279520648BF41F480418079C00648BF22
S11324A041F480510846704738B504460D46FFF79D
S11324B0D9FF00F030F8A87A10B1022804D00DE05A
S11324C0E8884000207009E0E888400020702889EE
S11324D04000E071607940F008006071A078A9784C
S11324E000F0FD0040EA4100297840EAC110A070E4
S11324F06079297900F06F0040EA0110697840EAB8
S1132500C110E97800F001F831BD00F0DF0040EAC5
S11325104110607170470FF23C0151F820007FE7D1
S113252010B504460021FFF794FF2046FFF79AFFF9
S11325300FF2200151F82000BDE810407CE7002193
S1132540817241708170C170017101210170704705
S1132550006006400600341000210FF2501252F8B9
S11325602130834202D0491C0229F8D3084670471F
S1132570F8B50D46044628680101B2FBF1F6B6B27F
S113258006B901265301B3FBF1F1A1EB4617510043
S1132590720112FA87F2B1FBF2F1091A6422B0FB5C
S11325A0F2F000EB4000884202D240F2F530F2BD76
S11325B02046FFF7D1FF00F043F81043086007F00E
S11325C01F01E07800F0F300E070207800F0E000F4
S11325D040EA262020706670A07A00F0E0000843EC
S11325E0A072A078297900F0EC000843A070687903
S11325F0E074A8796075207C40F088002074607CC9
S113260040F0C0006074E078E97909B140F0080056
S1132610297A09B140F00400E0700020F2BD80B5D1
S1132620017D0029FCD101794906FCD50021C17046
S1132630FFF792FF00F004F822EA0000086001BDF1
S11326400FF2700151F82000010C01F1804101F5F5
S11326508E2101230A6803FA00F070474FF4E13138
S11326600160002101714171012181710021C17159
S11326700172704702780A430270C27842EA11225A
S1132680C270827942EA11428271427C42EA11614B
S11326904174704705E003791B06FCD511F8013B32
S11326A0C37113465A1E002BF5D1704700A0064093
S11326B000B006400A0034100B0034100029817861
S11326C014BF41F0800101F07F018170704710B5A3
S11326D0644C82B02046FFF7DAFE00F01201E1708C
S11326E000F05001102911D041065F4A14D540076B
S11326F0A0780CD540F01000A07000208DF80000E8
S11327006846D16888479DF80000207113BD00F029
S1132710EF00A070207913BDA178C90603D5C007C6
S1132720EBD5A078F3E7207912690021904713BD17
S113273040684D49405C70474B498A6842B14A68D9
S113274013780370501C48608868401E8860704786
S11327500021017070474449496908475A2806D145
S1132760414A01238B54414911615169084770471B
S1132770FEB53D4D044669616068A2680221904738
S113278066680FF2F80050F826706846FFF7D7FE27
S11327901020ADF80600694635488068006990F855
S11327A07900FF2818BFADF806003846FFF77CFE15
S11327B001213846FFF782FF40213846FFF75AFED1
S11327C0FFF789FA4FF47A71B0FBF1F02949B1FBB4
S11327D0F0F0002100E011464A1C00FB02F3322B0A
S11327E0F9D321B9B0F5FA7F04D8012102E02029F8
S11327F028BF1F21B87900F0F0000843B871012107
S11328003046FFF775FC1C482861012061684919AE
S113281048700020FEBD70B50546134C6868011968
S11328204978A9B10FF2540151F820600021FFF753
S11328305FFC00213046FFF741FF3046FFF770FE92
S11328406868AA68002190476968091900204870DF
S113285070BD05484160826081680029FCD1002078
S11328607047000000600640540D00209F020020C5
S1132870E80C002040420F00A50200200060064042
S113288010B594488068006900F1680434214FF45D
S11328907070FFF73BFC48B934224FF47071204646
S11328A0FFF794FA20688C49884204D0FF2234212F
S11328B02046FFF733FAFFF72FFA002010BD38B592
S11328C0844DA86804694B20E07004F110020220D2
S11328D0A07004210020607020705020E07101205D
S11328E0A07102206071002020715420E072012048
S11328F0A0726072002020720120206340F64B50C9
S1132900606305F120002B69DB6A98472B69DB6A59
S113291004F11402012100F057F82B69DB6A04F179
S11329201802002100F050F82B69DB6A04F11C0244
S1132930022100F049F82B69DB6A04F1200203212B
S113294000F042F82B69DB6A04F14402052100F02F
S11329503BF82B69DB6A04F14802062100F034F8E5
S11329602B69DB6A04F14C02072100F02DF868683A
S11329700168A165E16500225849216658496166EC
S11329806969E26007E094F878501D4202D0E56876
S11329902B43E360521C182303FB02131B68002B18
S11329A0F1D150490A6822644A68E2638968A163E4
S11329B050F8101F616241680068081A401CA06248
S11329C001202065002032BD05F1200018470000D9
S11329D0F8B514463F4A444F91680426401E0969DD
S11329E017281D464BD8DFE800F00C121416181AED
S11329F0204A4A22242B4A1C1E2E313D4042444682
S1132A004A4805B12E6004B121600020F2BD0C31AA
S1132A10F7E71031F5E71431F3E71831F1E7203126
S1132A20EFE72431EDE72831EBE73431E9E73031E2
S1132A30E7E7D06941694969884738603946E0E782
S1132A4010265831DDE729480068F6E702F1200036
S1132A5012699269694690479DF800000028ECD0FD
S1132A600120EAE70C263831CBE74431C9E7483185
S1132A70C7E74C31C5E75031C3E70831C1E742F637
S1132A803C00F2BD134A92681369401E062842F6C0
S1132A903E0218D909380AD0401E012884BFC01E3E
S1132AA0032810D9083808D0801E0CD00EE0002965
S1132AB018BF012903D119637047032901D31046B4
S1132AC070471965704742F63D00704742F63C0076
S1132AD070470000E80C00206B63666700E0FF1F8E
S1132AE0A711002058800440000F002024800440D7
S1132AF030B5044685B060686946FEF77DF888BB4A
S1132B006068012814BF3B4D3B4D01A8FFF7A6FDAB
S1132B100098019001208DF80B008DF80C0060687E
S1132B20FFF7E7F8024601A92846FFF721FDB0B9EF
S1132B3060680121FFF700FB4FF400512846FFF7BE
S1132B4099FD6068A2682D4C0221904761685A2063
S1132B5088476168A62088470120207003E06068E8
S1132B60FEF730F8002005B030BD10B50446234808
S1132B7041606068A268012190476068FEF722F80E
S1132B80002010BD10B504461C48007850B16068A0
S1132B900021FFF7D1FA6068012814BF15481648D0
S1132BA0FFF73DFD6068FEF725F86068A268BDE8A0
S1132BB010400021104780B54068012814BF0D481B
S1132BC00D48FFF767FD002002BD0D480178890616
S1132BD000D50AE070470B4801788A0701D5C07810
S1132BE07047890600D500E07047C07803494968FA
S1132BF00847000000A0064000B00640040F002073
S1132C0004A0064004B00640AF49D1F88820531C04
S1132C105218C1F8883082F82000D1F8880000F0FA
S1132C203F00C1F88800704700207047B8E02DE9E4
S1132C30FC410C00154614BF002D0420984628D0F2
S1132C40A14F002007F190062860707000F0A8F8EA
S1132C5018B11EE0A22000F075F820213846FEF7D6
S1132C605BFB42463946684600F0F8F810B1002193
S1132C7029600EE03946684600F042F9BDF80410B8
S1132C808142E7D1012030702760BDF8020028603E
S1132C900020BDE8F6812DE9F0410C0082B0154614
S1132CA01E4635D0212D33D200F07AF800283FD1CA
S1132CB0DFF8148298F8910010B1002088F8910090
S1132CC008F160075A203870A42078700EB1A5204E
S1132CD078707D802DB12A46214608F16600FFF701
S1132CE065F808F16601384600F00AF9B880A91DB4
S1132CF0384600F064F8D8B9684600F0EFF8B8B97F
S1132D009DF80100A12812D0A22806D0A32801D042
S1132D1004200DE042F212700AE07888811D3846E2
S1132D2000F04DF820B99DF80100A228E4D000205D
S1132D30BDE8F6816548012181700021017070476A
S1132D402020704780B55A218DF800108DF80100BD
S1132D5001205D4981F891000221684600F02FF8B6
S1132D6002BD10B50446594882B001784278807893
S1132D701140014211D10FF2B8100088ADF80000E3
S1132D80022223695B6869462046984723690FF24B
S1132D90A4115B6808222046984742F2137016BDBE
S1132DA04A48017819B100210170A12004E081781A
S1132DB019B100218170A320C4E700207047444A60
S1132DC0D3690A46014618461B695B6818472DE912
S1132DD0F14F8B461646FDF794FF04464FF47A7084
S1132DE088467043FDF79DFFDFF8DCA00027064608
S1132DF089460AF188050EE06868296888420CD083
S1132E005044009990F8200078547F1C6868401C56
S1132E1000F03F0068605F451DD0FDF772FF021BA4
S1132E2061EB080341450AD828BFA04207D2E24318
S1132E306FEA080310185941421C41F10003B9F12B
S1132E40000F08BF002ED7D04B45D5D301D8B242CE
S1132E50D2D3052000E00020BDE8F28F70B582B027
S1132E6005460C46164600F039F858BB6878A62883
S1132E7004D11748C069FFF774FF76BDA42106B1D9
S1132E80A521884201D0012076BD00F023F8BDF8C9
S1132E9000106980B0B908462128A8BF20206880A6
S1132EA000F018F8BDF80010A98058B9698849B134
S1132EB02046FFF76DF869880A2000FB01F22046DE
S1132EC0FFF785FF76BD00000C0F00209C0F00204B
S1132ED0E80C002014220221684678E710B5044665
S1132EE0002201212046FFF772FF40B920785A28BA
S1132EF0F6D1601CBDE810400A22012167E710BD2D
S1132F0030B583B004460D46684600F017F8042235
S1132F102146684600F015F862882946684600F0A4
S1132F2010F801A9684600F023F8BDF804003EBD7E
S1132F305AA70000000201500000AAEA0021018003
S1132F40704770B5038800240EE0655C83EA0523AE
S1132F5008255E001B0444BF86F4805686F02106D3
S1132F606D1E3346F5D1641C9442EED3038070BDCC
S1132F70008808807047000005484CF22051C18148
S1132F804DF62811C1814FF4E9710180704700BFEB
S1132F900020054000F00BF8002801D000F00AF8EA
S1132FA00020C046C046FEF777FBFEF7B7FB0120C2
S1132FB07047000010B5074979441831064C7C4429
S1132FC0163404E00A68081D511888470146A142D6
S1132FD0F8D110BDAC010000B801000045EAFF1FA4
S1132FE053EAFF1FECE4FF1FF80D002034E6FF1F37
S1132FF06C0D0020C4E6FF1FD80C00207CE5FF1FE9
S113300064E6FF1F00000000000000000000000054
S113301000000000000000000000000000000000AC
S1133020000000000000000000000000000000009C
S1133030000000000000000000000000000000008C
S1133040000000000000000000000000B9FCFF1FA9
S1133050D7FCFF1F0000000000000000000000007B
S11330600000000081020020A502002000000000F2
S113307000000000FFFF01000100000004E6FF1F44
S113308000E0FF1FFF1F0020010000004CE6FF1FAF
S113309000000040FFFF074000000000D4E5FF1FD0
S11330A000F00F40FFFF0F4000000000D4E5FF1FB9
S11330B0000000E0FFFF0FE000000000D4E5FF1F68
S11330C000000000000000000000000000000000FC
S11330D00000400130B504E012F8014B00F8014B48
S11330E0491ED1B1C507F7D40129F5D0850701D40C
S11330F0042904D232F8024B20F8024B891E8B08B3
S1133100EFD000EB830403E052F8045B40F8045B67
S1133110A042F9D3A1EB8301E3E730BD80B51346A8
S11331200246184600E080B5FFF7D4FF002002BD38
S1133130FFF7FEBFC046C046C046C046FFF72AFFA1
S113314019E050F8041BCB0744BFA9F10103591837
S1133150121F0023042A41F8043BF9D25FEA827C5F
S11331600B4604D54FF0000CA1F800C09B1CD107FE
S113317044BF0021197050F8042B002AE1D1704794
S1133180C1FFFFFFD4010000D00D002000000000AB
S113319062B38B0708D0521E11F8013B00F8013BC3
S11331A000F024808B07F6D1830740F0208000BF15
S11331B0103A07D330B4B1E83810103AA0E8381008
S11331C0F9D230BC530724BFB1E80810A0E80810B6
S11331D044BF51F8043B40F8043BD20724BF31F804
S11331E0022B20F8022B44BF0B7803707047083A77
S11331F007D3B1E80810083A40F8043B40F804CB80
S1133200F7D25307E4E7FEE780B518491848086089
S113321018491948421A194888421CBF002AFFF766
S1133220B7FF17481749091A18BF00F037F81649AD
S11332301648421A04D0BDE808401548FFF7A8BF55
S113324001BD14484FF0FF31016041608160C160ED
S1133250016141618161C1610F4801604160816028
S1133260C160016141618161C161704708ED00E0A5
S1133270000000000000000000000000000000004A
S113328000000000000000006C3300006C330000FC
S1133290001E002080E100E080E200E0002200F057
S11332A001B80000401810F0030308D0C91A1FD356
S11332B0DB0748BF00F8012D28BF20F8022D1300BA
S11332C030B414461546103928BF20E93C00FAD81A
S11332D0490728BF20E90C0048BF40F8042D8900A5
S11332E028BF20F8022D48BF00F8012D30BC7047DC
S11332F0C91818BF00F8012DCB0728BF00F8012D0D
S11333007047000005484CF22051C1814DF6281148
S1133310C1814FF4E9710180704700BF002005406E
S113332000F00BF8002801D0C046C0460020C0467B
S1133330C046FDF7BDF800F002F80120704700F028
S113334001B800000746384600F002F8FBE7000029
S11333502021090326311820ABBEF9E7FFF7FEBF91
S10F3360C046C046C046C046FFF7DAFF76
S9030411E7
